:020000040000FA
:030000000200916A
:03002B00020705C4
:10003B0002070653D9BF79012200000080FB120092
:10004B003EB9000302008BE49001A1783579018061
:10005B0002F0A3D8FCD9FA9001D5AA82AB83900009
:10006B00A078AD79018015E493A3AC82AD838A822D
:10007B008B83F0A3AA82AB838C828D83D8E9D9E7DB
:10008B001202D812004475D0007581BF7510A1758E
:10009B001101020049506C656173652077616974C9
:1000AB002E2E2E3F00444F4E4521204453313038E5
:1000BB0035207375636365737366756C6C79206338
:1000CB006F6E66696775726564213F00596F7520A5
:1000DB0063616E207475726E20706F776572206F1E
:1000EB0066663F004552524F5221204453313038FF
:1000FB0035204E4F5420636F6E6669677572656469
:10010B00213F00506C65617320636865636B2068E9
:10011B006172647761726520636F6E6E656374697B
:10012B006F6E733F00616E6420747279206167613A
:10013B00696E3F00010000000001000000A1860174
:10014B0000C008C3E096F50808A3E096420808A390
:10015B00E096420808A3E09645087001D3D0082228
:10016B00E026F608A3E036F608A3E036F608A3E08F
:10017B0036F622E0F608A3E0F608A3E0F608A3E0C3
:10018B00F6222510C582C0E0E51134FFC583C0E01F
:10019B00E510C3958224F910AF0885831185821071
:1001AB008008858311858210D2AFCEF0A3E520F0B5
:1001BB00A37808E608F0A3DEFAEFF0A3E58124FBB1
:1001CB00F8E608F0A3E608F0A30808E608F0A3E6B3
:1001DB0008F0A315811581D0E0FED0E0F81581154C
:1001EB0081E8C0E0EEC0E022851183851082E0A398
:1001FB00FEE0A3F5207808E0A3F608DFFAE0A3FF02
:10020B00E0A3C0E0E0A3C0E0E0A3C0E0E0A3C0E057
:10021B0010AF088582108583118008858210858335
:10022B0011D2AFD083D0822274F712018D89087559
:10023B00090074C22508F58274113509F583E4931E
:10024B009001A3F09001A3E0FA7B00EA75F008A4FB
:10025B00CAA8F075F000A428F875F008EBA428FBE9
:10026B009001A1EAF0A3EBF07F020201F375A40D5C
:10027B0075A5E775A70175D40F75D50775DF0175E2
:10028B00E10575E2422275B980780080020008E82A
:10029B00C3941440F843B9C0E5B9A2E550FA75A967
:1002AB000275B28322D28C438922438E0C758CB09B
:1002BB0075C18043E601221202911202781202B03C
:1002CB00C283D282D280C292D291D2AF2253D9BFF3
:1002DB001202C21208831208647AFF7BFF120A749F
:1002EB007CD57D017A827B007972120B669001A41A
:1002FB00E0D2E4F09001A57458F080079001A5E0DE
:10030B002401F09001A5E0C39460502F9001A774D5
:10031B0037F09001A4E0D2E3F09001A4E0D2E1F039
:10032B0012067D9001A4E0A2E440D19001A5E090DB
:10033B0001A6F09001A8E09001BAF09001AC740016
:10034B00F080079001ACE02401F09001ACE0C39485
:10035B000A400302044512055A9001A57459F01284
:10036B0004479001CCE0541FF09001B8E0541FF00B
:10037B009001D0E0540FF09001BCE0540FF09001CD
:10038B00AB7401F080079001ABE02401F09001AB5E
:10039B00E0C3941050449001ABE0640C60089001F2
:1003AB00ABE0640D70069001AB740EF09001ABE006
:1003BB00F8790074C128F582740139F583E0FA905D
:1003CB0001ABE0F8790074AD28F582740139F5833F
:1003DB00E06A60B29002747400F0900274E0640101
:1003EB00701C7CE57D017A0A7B007972120B667CAE
:1003FB000C7D027A1E7B00790F120B66803C9001FC
:10040B00ACE0C39407500302034E900274E0600308
:10041B0002034E7C247D027A327B007972120B66CA
:10042B007C437D027A0A7B007928120B667C657D02
:10043B00027A0A7B00790F120B6680FEC082C083A2
:10044B009001A77401F09001A4E0D2E3F09001A415
:10045B00E0D2E1F012067D9001A5E09001C1F09091
:10046B0001A7E09001C2F09001A8E09001C3F090C9
:10047B0001A9E09001C4F09001A77402F09001A4CF
:10048B00E0D2E3F09001A4E0D2E1F012067D9001FE
:10049B00A7E09001C5F09001A8E09001C6F0900193
:1004AB00A9E09001C7F09001A77408F09001A4E0B7
:1004BB00D2E3F09001A4E0D2E1F012067D9001A707
:1004CB00E09001C8F09001A8E09001C9F09001A95B
:1004DB00E09001CAF09001A7740EF09001A4E0D255
:1004EB00E3F09001A4E0C2E1F012067D9001A7E0D9
:1004FB009001CBF09001A8E09001CCF09001A77493
:10050B0037F09001A4E0D2E3F09001A4E0C2E1F057
:10051B0012067D9001A7E09001CDF09001A8E0902C
:10052B0001CEF09001A7740DF09001A4E0D2E3F09E
:10053B009001A4E0C2E1F012067D9001A7E09001CA
:10054B00CFF09001A8E09001D0F0D083D08222C0F0
:10055B0082C0839001A77401F09001A87400F09001
:10056B0001A97400F09001A4E0C2E3F09001A4E0B3
:10057B00D2E1F012067D9001A6E09001ADF0900162
:10058B00A7E09001AEF09001A8E09001AFF09001D0
:10059B00A9E09001B0F09001A77402F09001A8744B
:1005AB0018F09001A97400F09001A4E0C2E3F09060
:1005BB0001A4E0D2E1F012067D9001A7E09001B119
:1005CB00F09001A8E09001B2F09001A9E09001B386
:1005DB00F09001A77408F09001A874C3F09001A9E2
:1005EB007400F09001A4E0C2E3F09001A4E0D2E12A
:1005FB00F012067D9001A7E09001B4F09001A8E005
:10060B009001B5F09001A9E09001B6F09001A774AC
:10061B000EF09001BAE0131313541F9001A8F09041
:10062B0001A4E0C2E3F09001A4E0C2E1F012067D68
:10063B009001A7E09001B7F09001A8E09001B8F00D
:10064B009001A7740DF09001A87409F09001A4E03B
:10065B00C2E3F09001A4E0C2E1F012067D9001A785
:10066B00E09001BBF09001A8E09001BCF0D083D0EA
:10067B00822274F112018D900275780812017E901E
:10068B0001A4E0D2E0F0C2AD9001A4E0A2E35012CD
:10069B009001A4E0D2E2F09001A4E0C2E3F0D2C555
:1006AB00804B9001A4E0C2E2F0D2C5804085080CDB
:1006BB0085090D850A0E850B0F850C08850D09859F
:1006CB000E0A850F0B900279780812016B90027D50
:1006DB00780C12014C50169001A4E0A2E4500E903D
:1006EB0001A4E0C2E0F09001A4E0D2E4F09001A4F8
:1006FB00E0A2E040B87F080201F332C0E0C0D0E8CE
:10070B00C0E0E9C0E0C008C009C082C083A2C250EB
:10071B0003020848E5C075090054F0F8E5095400D8
:10072B00F9E8248070030207F624C0602124E060FE
:10073B00030208489001A5E0C333F5C253C2FE90F3
:10074B0001A4E0A2E3E43342C2C2C5020848A2C13D
:10075B0040030207EA9001A4E0C2E4F09001A4E098
:10076B00A2E350030208489001A4E0A2E1400E90DE
:10077B0001AAE0640270069001AA7403F09001AA2A
:10078B00E0600B146017146036146042805B9001BC
:10079B00AAE02401F09001A7E0F5C2804C9001A4DF
:1007AB00E0A2E2500B9001A4E0D2E3F0D2C5803975
:1007BB009001AAE02401F09001A8E0F5C2807E90A0
:1007CB0001AAE02401F09001A9E0F5C2806F90012D
:1007DB00A4E0C2E0F09001AA7400F0D2C4805E9055
:1007EB0001AA7400F0D2C4D2C580529001A4E0C219
:1007FB00E4F09001AAE014600514602C803FE5C280
:10080B009001A8F09001AAE02401F09001A4E0A2CD
:10081B00E14011C2C19001AA7400F09001A4E0C2A2
:10082B00E0F08019D2C18015E5C29001A9F0C2C1D8
:10083B009001AA7400F09001A4E0C2E0F0C2C0D015
:10084B0083D082D009D008D0E0F9D0E0F8D0D0D056
:10085B00E03275A60075A0FF2275A6FF22D2917A11
:10086B00057B00120BC1C2917A0A7B00120BC1D21D
:10087B00917A327B00020BC1D296D282D2921208AD
:10088B00641208687A027983120A0B7A037985124B
:10089B000A0B7A93798C120A0B7A017991120A0B53
:1008AB007A007983120A0B7AB0793E120A0B7A031B
:1008BB00793F120A0B7A107940120A0B7A5679415A
:1008CB00120A0B7A137942120A0B7A467943120AEF
:1008DB000B7A237944120A0B7A767945120A0B7A32
:1008EB00007946120A0B7A5E7947120A0B7A4F7916
:1008FB0048120A0B7A407949120A0B7A617917125E
:10090B000A0B7AF9792B120A0B7A0A7B00120BC1AC
:10091B007A14791B120A0B7A11791A120A0B7A0DB7
:10092B00791C120A0B7A3D791F120A0B7A147B0081
:10093B00120BC17A0A7919120A0B7A1A7919120A4F
:10094B000B7A287B00120BC17A127919120A0B7AD7
:10095B00287B00120BC17A20791E120A0B7A647B5A
:10096B0000120BC17A60793C120A0B7A40793D1266
:10097B000A0B7A387934120A0B7A387935120A0B4A
:10098B007A387924120A0B7A287B00120BC17A3C35
:10099B007924120A0B7A1C7916120A0B7A06790142
:1009AB00120A0B7A007955120A0B7A007902120A95
:1009BB000B7A007903120A0B7A007904120A0B7A6C
:1009CB00EF7905120A0B7A007906120A0B7A007975
:1009DB0007120A0B7A017908120A0B7A8F7909121E
:1009EB000A0B79221209F502085DD283C29289A003
:1009FB00C280D280D292C2832289A0C280D28022AE
:100A0B00D283C29289A0C280D280D2928AA0C280A5
:100A1B00D280C2832274F812018DEAFEEBFFD283DF
:100A2B00EEF8EFF9E4E9F8F9120A04EEF9120A0408
:100A3B00C2837F010201F374F812018D8908EAFE6B
:100A4B00EBFF120864AA087903120A0BEEFAEFFB0C
:100A5B00E4EBFA7906120A0BEEFA7907120A0B7914
:100A6B00221209F57F010201F374F712018DEAFEE0
:100A7B00EBFFD2961208647A007B007900120A42CF
:100A8B0079221209F57508F97509C0EEFAEFFB1218
:100A9B000A20EEFAEFFB120A20A80874FF28F508CB
:100AAB00E870E8A90974FF29F509E970DE7F0202F5
:100ABB0001F374F112018D89088A0E8B0F8C09A931
:100ACB0009120233750C008002050CE50CC3940867
:100ADB004003020B61850C0A750B00E50E250AFA23
:100AEB00E50F350BFBA908120A427E007F20792205
:100AFB001209F5750D0080107AFF7BFF120A20EFAB
:100B0B00C313FFEE13FE050DE50DC3940E50BA9003
:100B1B0001A1850C0A750B00E0250AF8A3E0350B43
:100B2B00F9E875F002A4C8AAF075F000A42AFA75CA
:100B3B00F002E9A42AF974C228F582740B39F58303
:100B4B00E4935EF8A3E4935FF9E84960AB7A007B2A
:100B5B00F8120A2080A97F080201F374F312018DA9
:100B6B0089088A0C8B0D8C0A8D0B7E007F008026EA
:100B7B00EEF8EFF9E875F00AA4C8AAF075F000A436
:100B8B002AFA75F00AE9A42AF9E8250CFAE9350DD9
:100B9B00FBA908120ABDE50A2EF582E50B3FF5838A
:100BAB00E0F8EE2401FEEF3400FFE8FC743F6870C0
:100BBB00BF7F060201F322000000000000000000CE
:100BCB0000000000000000000000000000FF33FFE9
:100BDB0033000000000000000007000700000000C9
:100BEB00000700070000002001FE1FFE1F20012050
:100BFB0001FE1FFE1F200138063C0E6408FF3FFF5D
:100C0B003F84091C0F18071E30331C1E07C00170D0
:100C1B00001C1E0733011E1E1FB331E120E120B360
:100C2B00311E1F001B80310000000000000B00076D
:100C3B000000000000000000000000F807FF3F0765
:100C4B003800000000000000000000000000000061
:100C5B000000000000000000000000000000000089
:100C6B000000000000000000000000000000000079
:100C7B000000000000000000000000000000000069
:100C8B000000000000000000000000000000000059
:100C9B000000000000000000000000000000300019
:100CAB00300000000000000030003C000FC003F0DB
:100CBB00003C000F000300FC0FFE1F033681216177
:100CCB00201B30FE1FFC0F042004200620FF3FFFDB
:100CDB003F0020002000200C380E3C03260123810E
:100CEB0021C3207E203C20061803304120412041A7
:100CFB00204120E330BE1F000FE00FFC081F0883CC
:100D0B003F803F000800083F0C3F1C213021202171
:100D1B00206130C11F810FE00FF81F5C304620436C
:100D2B0020C130811F010F010001000100013C8136
:100D3B003FF1037F000F001C0FBE1FE3304120412A
:100D4B0020E330BE1F1C0F3C207E20C3208130814E
:100D5B0018830EFE07FC01000000000000000000DD
:100D6B000000000000000000000000000000000078
:100D7B000000000000000000000000000000000068
:100D8B0000000000000000200120012001200120B4
:100D9B0001200120012001000000000000000000E4
:100DAB000000000000000000000000000000000038
:100DBB000000000000000000000000000000000028
:100DCB0000000000000000FC3FFE3F030101010199
:100DDB00010301FE3FFC3FFF3FFF3F41204120410C
:100DEB0020E330BE1F1C0FFC0FFE1F033001200140
:100DFB002003300E1C0C0CFF3FFF3F012001200194
:100E0B00200738FE1FF807FF3FFF3F4120412041DD
:100E1B0020412041200120FF3FFF3F8100810081C5
:100E2B0000810081000100FC0FFE1F0330012081B7
:100E3B002083308E1F8C0FFF3FFF3F400040004050
:100E4B00004000FF3FFF3F012001200120FF3FFF3B
:100E5B003F012001200120000C001C00300020006D
:100E6B00200030FF1FFF0FFF3FFF3FC000E00138A6
:100E7B00071C0E0F3C0330FF3FFF3F0020002000FC
:100E8B0020002000200020FF3FFF3F7800C003C060
:100E9B00037800FF3FFF3FFF3FFF3F1C007000C088
:100EAB00010007FF3FFF3FFC0FFE1F033001200136
:100EBB00200330FE1FFC0FFF3FFF3F8100810081AD
:100ECB0000C3007E003C000000000000000000009A
:100EDB0000000000000000FF3FFF3F810081008108
:100EEB0001C31F7E3E3C203C0C7E1C6330E120C1C5
:100EFB002183318E1F0C0F030003000300FF3FFF04
:100F0B003F030003000300FF0FFF1F003000200012
:100F1B00200030FF1FFF0F3F00FF01C00F003C0000
:100F2B003CC00FFF013F00FF01FF3F003EC001C06F
:100F3B0001003EFF3FFF0100000000000000000029
:100F4B00000000000000003F00FF00C001803F8058
:100F5B003FC001FF003F000138013E8127C12161E5
:100F6B002039201F20072000000000000000000097
:100F7B000000000000000000000000000000000066
:100F8B000000000000000000000000000000000056
:100F9B000000000000000000000000000000000046
:100FAB000000000000000000000000000000000036
:100FBB000000000000000000000000000000000026
:100FCB0000000000000000001E403F2021202120D7
:100FDB00212011E03FC03FFF3FFF3F40102020206A
:100FEB00206030C01F800F800FC01F60302020207A
:100FFB0020202060304010800FC01F603020202048
:10100B00204010FF3FFF3F800FC01F603220222087
:10101B00226022C033801320002000FE3FFF3F21BF
:10102B00002100230002008007C00F601820102051
:10103B00104008E03FE03FFC3FFC3F400020002019
:10104B00006000C03F803F000020202020E33FE3F2
:10105B003F00200020000000000000000000000006
:10106B0000000000000000FC3FFC3F000600078072
:10107B000DC01860302020000001200120FF3FFF31
:10108B003F002000200000E03FE03F6000C01FC099
:10109B001F6000E03FC03FE03FE03F4000200020EA
:1010AB00006000C03F803F800FC01F6030202020B9
:1010BB00206030C01F800FE03FE03F40042008203D
:1010CB0008600CC007800300000000000000000057
:1010DB0000000000000000E03FE03FC00040006067
:1010EB0000600060004000C010E031202120232070
:1010FB00262024603C4018000020002000FE1FFE2C
:10110B003F202020200000E01FE03F0020002000B7
:10111B00200010E03FE03FF003F007001C00300020
:10112B0030001CF007F003E007E03F0038E007E079
:10113B00070038E03FE0070000000000000000005F
:10114B0000000000000000E001E02700260038004E
:10115B0018000EE007E00120302038202C2026203C
:10116B0023A021E020602000000000000000000010
:10117B0000000000000000000000000000FF3FFF27
:10118B003F00000000000000000000000000000015
:10119B000000000000000000000000000000000044
:1011AB000000000000000000000000000000000034
:1011BB000000000000000000000000000000000024
:1011CB000000000000000000000000000000000014
:1011DB0000000000000000000102030405060708E0
:1011EB00090A0B0C0D0E0F101112131415161718EC
:1011FB00191A1B1C1D1E1F202122232425262728DC
:10120B00292A2B2C2D2E2F303132333435363738CB
:10121B00393A3B3C3D3E3F404142434445464748BB
:10122B00494A4B4C4D4E4F505152535455565758AB
:10123B00595A5B5C5D5E5F0000000000000000001F
:10124B000000000000000000000000000000000093
:10125B000000000000000000000000000000000083
:10126B000000000000000000000000000000000073
:10127B000000000000000000000000000000000063
:10128B000000000000000000000000000000000053
:10129B000000000000000000000000000000000043
:1012AB000000000000000000000000000000000033
:0712BB00000000000000002C
:040000050000009166
:00000001FF
